:1000000091C00000ACC00000AAC00000A8C0000061
:10001000A6C00000A4C00000A2C00000A0C0000054
:100020009EC000009CC0000085C3000044C30000C7
:1000300096C0000094C0000092C0000090C0000074
:100040008EC000008CC000008AC0000088C0000084
:1000500086C0000084C0000082C0000080C0000094
:100060007EC000007CC000007AC0000078C00000A4
:1000700076C0000074C0000072C0000070C00000B4
:100080006EC000006CC000006AC0000068C00000C4
:1000900066C0000064C000001201100102000008E8
:1000A000EB03442001000102DC0109023E000201D1
:1000B00000C0320904000001020201000524001002
:1000C0000104240206052406000107058203080036
:1000D000FF09040100020A000000070504021000E5
:1000E00005070583021000050403090418034400F2
:1000F000650061006E002000430061006D00650036
:100100007200610000001C034C00550046004100D5
:1001100020004300440043002000440065006D00BF
:100120006F00000011241FBECFEFD0E2DEBFCDBFB5
:1001300011E0A0E0B1E0EAE6FFE000E00BBF02C0A2
:1001400007900D92AE36B107D9F711E0AEE6B1E0F7
:1001500001C01D92AA38B107E1F777D004C750CF8C
:100160008BB18F70806A8BB908958BB18F7080616D
:100170008BB90895089582E591E01DC682E591E06E
:10018000F3D580FD02C090E901C090E68BB18F707D
:10019000982B9BB9089523B18CB1809590E0807322
:1001A0009070959587952095207E282B27FD17C068
:1001B00024FF03C020E031E014C026FF03C020E18B
:1001C00031E00FC023FF03C020E231E00AC025FF69
:1001D00003C021E331E005C010926E01089524E4CC
:1001E00031E080916E01882339F481E080936E01C3
:1001F000C9016FE671E08CC6089584B7877F84BF1C
:1002000088E10FB6F89480936000109260000FBEF2
:1002100080E090E020E80FB6F8942093610080938E
:1002200061000FBE84B18F7184B98DB18F7C8DB99F
:1002300085B1806E85B98EB180638EB98AB1806FC9
:100240008AB98BB18F708BB91BC2D7DF82E591E081
:100250006FE671E0EED48BB18F7080618BB97894CA
:100260009ADF82E591E0B3D482E591E030D59AD46B
:10027000F7CFDA01923049F0933061F09130F9F420
:10028000E8E9F0E022E130E01EC0EAEAF0E02EE327
:1002900030E019C0813049F0813018F0823079F4B3
:1002A00008C0E8EEF0E0849107C0ECEEF0E0849145
:1002B00003C0E6E0F1E08491282F30E004C0E0E0E4
:1002C000F0E020E030E0ED93FC93C90108959C013B
:1002D00040918801509189014617570718F4F90198
:1002E00090E03DC06115710511F0AB01F8CF809130
:1002F000E8008E778093E80040E050E0F0CF8091F6
:100300008101882309F441C0853009F440C08091FF
:10031000E80083FD3EC08091E80082FD30C08091FE
:10032000E80080FF1CC02091F2003091F30007C06C
:1003300081918093F100415050402F5F3F4F411514
:10034000510519F02830310598F390E02830310537
:1003500009F491E08091E8008E778093E8004115E0
:10036000510569F6992359F60AC0809181018823C5
:1003700061F0853061F08091E80083FD0AC08091D2
:10038000E80082FFF2CF80E0089582E0089583E0E4
:10039000089581E008959C01409188015091890160
:1003A0004617570718F4F90190E03EC06115710532
:1003B00011F0AB01F8CF8091E8008E778093E800D0
:1003C00040E050E0F0CF80918101882309F442C0E1
:1003D000853009F441C08091E80083FD3FC08091E1
:1003E000E80082FD31C08091E80080FF1DC02091AF
:1003F000F2003091F30008C084918093F1003196AF
:10040000415050402F5F3F4F4115510519F02830A2
:10041000310590F390E02830310509F491E08091A6
:10042000E8008E778093E8004115510561F6992325
:1004300051F60AC080918101882361F0853061F016
:100440008091E80083FD0AC08091E80082FFF2CF2E
:1004500080E0089582E0089583E0089581E00895A2
:10046000382F282F2EC0822F8F708093E9002317FA
:1004700021F4762F942F50E006C07091EC009091FB
:10048000ED005091F00091FF1BC08091EB008E7F3A
:100490008093EB008091ED008D7F8093ED00809143
:1004A000EB0081608093EB007093EC009093ED0083
:1004B0005093F0008091EE0087FD02C080E0089527
:1004C0002F5F273080F23F703093E90081E008957C
:1004D0000F931F93CF93DF93062FEC0110E02AC0F8
:1004E0009881992329F16B81E981FA812C81892FE7
:1004F0008F70873018F5223010F452E001C056E0BA
:1005000040E028E030E003C04F5F220F331F2E177A
:100510003F07D0F36295660F660F607C991F99279D
:10052000991F692B4295407F452B9ADF882331F034
:100530001F5F25961017A0F281E001C080E0DF91D7
:10054000CF911F910F9108958091820188239CF48F
:1005500004C0809181018823B9F08091E80082FF76
:10056000F8CF8091E8008B778093E8000895809120
:100570008101882349F08091E80080FFF8CF8091C5
:10058000E8008E778093E80008954091E400509150
:10059000E50024E68091EC0080FF24C08091E80013
:1005A00080FD1EC080918101882311F482E00895AE
:1005B000853011F483E008958091EB0085FF02C03F
:1005C00081E008958091E4009091E50084179507FB
:1005D00009F3222311F484E008952150AC01DACF0D
:1005E00080E008958091E80082FFDCCFF9CFEF92A0
:1005F000FF920F931F9352D059D008ED10E0F801ED
:1006000080818F77808380818068808380818F7DE7
:100610008083E7EDF0E080818068808319BC1092D0
:10062000810110927D0110927F0110927E0180EE77
:10063000E82EF12CF70180818B7F8083F801808187
:100640008160808380E060E042E00ADFE1EEF0E07C
:1006500080818E7F8083E2EEF0E080818160808304
:10066000808188608083F70180818E7F8083F8019C
:100670008081806180831F910F91FF90EF9008959A
:10068000E8EDF0E080818F7E8083E7EDF0E080810F
:100690008160808381E080938001A9CFE8EDF0E064
:1006A00080818C7F80831092E20008951092DA009E
:1006B0001092E10008951F920F920FB60F920BB6A1
:1006C0000F9211241F932F933F934F935F936F9338
:1006D0007F938F939F93AF93BF93EF93FF9310916B
:1006E000E9008091EC001092E9008091F000877F92
:1006F0008093F0007894EDD01092E9008091F000A2
:1007000088608093F0001F701093E900FF91EF91D3
:10071000BF91AF919F918F917F916F915F914F9119
:100720003F912F911F910F900BBE0F900FBE0F9016
:100730001F9018951F920F920FB60F920BB60F9243
:1007400011242F933F934F935F936F937F938F93D6
:100750009F93AF93BF93EF93FF938091E10082FF4C
:100760000AC08091E20082FF06C08091E1008B7F89
:100770008093E10016D28091DA0080FF1DC0809145
:10078000D80080FF19C08091DA008E7F8093DA0054
:100790008091D90080FF0CC08CE089BD8EE089BDBE
:1007A00009B400FEFDCF81E080938101D9DC04C053
:1007B00019BC10928101D9DC8091E10080FF18C042
:1007C0008091E20080FF14C08091E2008E7F8093D0
:1007D000E2008091E20080618093E2008091D80085
:1007E00080628093D80019BC85E080938101D9D1C3
:1007F0008091E10084FF2FC08091E20084FF2BC034
:100800008CE089BD8EE089BD09B400FEFDCF8091EA
:10081000D8008F7D8093D8008091E1008F7E8093F7
:10082000E1008091E2008F7E8093E2008091E200FF
:1008300081608093E20080917D01882311F084E043
:1008400007C08091E30087FD02C081E001C083E022
:1008500080938101A6D18091E10083FF27C0809120
:10086000E20083FF23C08091E100877F8093E10055
:1008700082E08093810110927D018091E1008E7F62
:100880008093E1008091E2008E7F8093E20080916E
:10089000E20080618093E20080E060E042E0E0DD21
:1008A0008091F00088608093F0007BD1FF91EF9100
:1008B000BF91AF919F918F917F916F915F914F9178
:1008C0003F912F910F900BBE0F900FBE0F901F9076
:1008D00018951F93DF93CF93CDB7DEB7AC970FB6C4
:1008E000F894DEBF0FBECDBFE2E8F1E08091F100E9
:1008F000819321E0EA38F207C9F73DDC8091E800F6
:1009000083FF37C18091820130918301353009F432
:1009100087C0363040F43130C9F1313070F03330B7
:1009200009F027C133C0383009F4F5C0393009F473
:1009300004C1363009F01DC196C0803821F08238DC
:1009400009F017C108C090917E0180917F01882332
:1009500099F0926011C0809186018F708093E900B8
:100960008091EB0090E025E0969587952A95E1F738
:10097000982F91701092E9008091E800877F809312
:10098000E8009093F1001092F100D0C0882319F094
:10099000823009F0EEC090E08F719070009721F0E6
:1009A000029709F0E6C00CC080918401813009F003
:1009B000E0C010927F01333069F580937F012AC037
:1009C00080918401882331F5209186012F7009F4EC
:1009D000D0C02093E9008091EB0080FF1BC0333032
:1009E00021F48091EB00806213C08091EB00806164
:1009F0008093EB0081E090E002C0880F991F2A9558
:100A0000E2F78093EA001092EA008091EB008860A0
:100A10008093EB001092E9008091E800877F89C005
:100A2000882309F0A6C0109184011F778091E3000C
:100A30008078812B8093E3008091E800877F80930A
:100A4000E80082DD8091E80080FFFCCF8091E30028
:100A500080688093E300112311F482E001C083E0F9
:100A60008093810186C08058823008F082C08091D6
:100A700084019091850123E08C3D920709F033C0F9
:100A800083E08C838AE28B837FB7F894DE0115962E
:100A90006EE040E050E011E2E62FF0E010935700E6
:100AA000849140FF03C082958F706F5F8F70282FF5
:100AB00030E08A3018F0C901C79602C0C901C0965B
:100AC0008D939D934F5F5F4F4431510529F77FBF51
:100AD0008091E800877F8093E800CE0103966AE268
:100AE00070E0F5DB12C060918601AE014F5F5F4F91
:100AF000C0DBBC01009709F43CC08091E800877F0F
:100B00008093E80089819A8146DC8091E8008B77A8
:100B10008093E8002EC0803861F58091E800877FDF
:100B20008093E80080917D018093F1008091E8003E
:100B30008E778093E80008DD1CC08823D1F4909163
:100B400084019230B0F48091E800877F8093E800C0
:100B500090937D01F9DC80917D01882331F48091AF
:100B6000E30087FD02C081E001C084E08093810141
:100B700005DB8091E80083FF0AC08091E800877F51
:100B80008093E8008091EB0080628093EB00AC964C
:100B90000FB6F894DEBF0FBECDBFCF91DF911F918E
:100BA000089508951F9380918101882371F0109119
:100BB000E9008091EC001092E9008091E80083FF49
:100BC00001C087DE1F701093E9001F910895FC019A
:100BD00080918101843049F584899589A689B789F6
:100BE0000097A105B10509F186818F708093E90016
:100BF0008091E80082FF19C08091F2009091F3008B
:100C0000892B19F42FEF3FEF04C08091F100282FBA
:100C100030E08091F2009091F300892B41F48091B3
:100C2000E8008B778093E80002C02FEF3FEFC90107
:100C30000895FB012EE0DB011D922A95E9F723E0E0
:100C4000238325EA36E0318720872CE236E033879C
:100C50002287958784870895FC0184859585B7DF71
:100C60009C0197FF02C02EEF3FEFC9010895089540
:100C7000FC0180918101843029F584899589A689B8
:100C8000B7890097A105B105E9F081818F70809344
:100C9000E9008091F2009091F300892BA9F09091E6
:100CA000E8008091E8008E778093E80095FD0CC005
:100CB0006CDC982F882349F48091E8008E7780932C
:100CC000E80003C092E001C090E0892F0895FC0184
:100CD00080918101843091F484899589A689B789AE
:100CE0000097A105B10551F081818F708093E900D3
:100CF0008091E80080FF02C0CF01BACF08951F9312
:100D0000FC01162F809181018430E1F4848995895A
:100D1000A689B7890097A105B105A1F081818F70DF
:100D20008093E9008091E80085FD08C08091E8008B
:100D30008E778093E80029DC882329F41093F10052
:100D400080E001C082E01F910895282FFB01848577
:100D50009585622FD4DF882319F420E030E002C0AB
:100D60002FEF3FEFC9010895CF93DF93EC01409639
:100D7000FC018BE0DF011D928A95E9F782E08C830C
:100D8000898783E08E87CE01019661E0A1DB88230D
:100D900071F0CE01069661E09BDB882341F0CE0125
:100DA0000B9661E095DB882319F081E001C080E0BB
:100DB000DF91CF910895CF93DF93EC018091E8000C
:100DC00083FFA3C0888190E0209186013091870144
:100DD0002817390709F099C080918301813269F0A1
:100DE000823220F4803209F090C03CC0823209F493
:100DF0006BC0833209F089C07AC080918201813A48
:100E000009F083C08091E800877F8093E80080919B
:100E1000E80080FFFCCF8C899D89AE89BF898093D3
:100E2000F100292F3A2F4B2F55272093F1009D01D8
:100E3000442755272093F1008B2F9927AA27BB27FA
:100E40008093F100888D8093F100898D8093F1006B
:100E50008A8D8093F1008091E8008E778093E8007E
:100E600073DB53C080918201813209F04EC08091C2
:100E7000E800877F8093E80005C080918101882386
:100E800009F443C08091E80082FFF7CF8091F10020
:100E90009091F1002091F1003091F1008C8B9D8BAD
:100EA0002E8B3F8B8091F100888F8091F100898F8C
:100EB0008091F1008A8F8091E8008B778093E80021
:100EC00043DBCE01D4DE21C0809182018132E9F47E
:100ED0008091E800877F8093E80036DB8091840171
:100EE00090918501998B888BCE0144D90EC0809159
:100EF0008201813251F48091E800877F8093E8007D
:100F000023DBCE0160918401B2DEDF91CF910895A1
:100F1000EF92FF920F931F93CF93DF937C018B018E
:100F2000DB0113968C9181FD03C0CFEFDFEF13C07F
:100F3000C0E0D0E00BC0D8011896ED91FC91199754
:100F4000B8010995892B11F0CFEFDFEFF7018191FF
:100F50007F01882381F7CE01DF91CF911F910F91FF
:0A0F6000FF90EF900895F894FFCF82
:100F6A004A6F79737469636B20446F776E0D0A0058
:100F7A004A6F79737469636B204C6566740D0A0055
:100F8A004A6F79737469636B2052696768740D0AD2
:100F9A00004A6F79737469636B2050726573736565
:100FAA00640D0A004A6F79737469636B2055700D7A
:100FBA000A000083100000010410000001820800EA
:0E0FCA00000100000000000000000000000018
:00000001FF
